:2000000021C03AC039C038C037C036C035C034C033C032C031C0D5C42FC02EC02DC02CC019
:200020002BC02AC0E3C6B1C6D0C626C025C024C023C022C071C5E7C456C56EC575C59DC5F6
:20004000ACC5C0C511241FBECFEFD2E0DEBFCDBF11E0A0E0B1E0EAE8FEE002C005900D9257
:20006000A030B107D9F711E0A0E0B1E001C01D92A030B107E1F701C0C3CFCFEFD2E0DEBFF6
:20008000CDBF1A9901C041C7E4D1F8D1A9D276D28093FC0122D2109287017894A0E0B0E0CD
:2000A000ECD6802D992780939101809191018F3F19F485E080939101BCD25F9841E150915C
:2000C000F10E752F7F718091C1018823E1F31092C1011092C2011092F20120E02093F30136
:2000E0001A9BFECF429A1A99FECF42988091F501882309F445C01092F5018091F701882348
:2001000049F11092F7018091020180FF0CC08091020182FF2BC08091020181FF23C08091A4
:20012000F20182600BC08091020181FF17C08091020182FF1FC08091F20181608093F20155
:200140008091F20184608093F20122E882E28093F40118C08091020180FF08C080910201F4
:2001600082FF0EC08091F201826007C08091020181FF06C08091F20181608093F20122E03C
:200180004093F4018091F601882341F01092F60128608091F20188608093F2018091F80196
:2001A000882331F028608091F20180618093F2018091850187FF58C028608091F201886057
:2001C0008093F201809185018038B9F48091F00E8093FD01852F807E8093FE018091FE0129
:2001E000872B8093FE018091F20E8093FF018091F30E8093000281E819C08091850181385E
:20020000D9F48091F40E8093FD018091F50E9091F60E892F99278093FE018091F50E809303
:20022000FF018091F70E8093000282E8809385011BC01092F10147CF809185018238A1F425
:200240008091F80E8093FD018091F90E9091FA0E892F99278093FE018091F90E8093FF0180
:200260008091FB0E809300022EBD40980DB407FEFDCF61E01A99C5C0409A8091C20187311B
:2002800098F48091F101882339F08091C201E82FFF27ED53FE4F06C08091C201E82FFF2786
:2002A000E652FE4F8EB580838091C2018F5F8093C2019091F301992309F044C08091F20109
:2002C00082FF1CC08091F20180FF0CC08091C201823120F18091C201E82FFF27E850FF4F43
:2002E000808123C08091C201823160F08091C201E82FFF27E050FF4F878517C08091F201CD
:2003000080FF08C08091C201E82FFF27E050FF4F81850BC08091F20181FF09C08091C20115
:20032000E82FFF27E050FF4F80A18EBD01C09EBD9091C2018091F401981709F061C06093D4
:20034000F3015EC08091F3018130C9F58091F20183FF1FC08091850187FF07C08091C201FA
:20036000E82FFF27E551FE4F11C08091F20182FF07C08091C201E82FFF27ED51FF4F06C03D
:200380008091C201E82FFF27EC50FF4F80818EBD01C01EBC8091C201282F33278091F40150
:2003A000992704962817390759F582E08093F30180918501823821F51092850121C080912C
:2003C000F3018230F1F48091F20184FF0AC08091F8018EBD8091F801813021F01092F80185
:2003E00001C01EBC8091C201282F33278091F401992705962817390719F483E08093F30186
:2004000040980DB407FEFDCF8091F301833009F031CF409A8091C201873198F48091F101CC
:20042000882339F08091C201E82FFF27ED53FE4F06C08091C201E82FFF27E652FE4F8EB5AB
:2004400080838091F101882309F0F3CE6093F1013ACE80E285B983E184B981E388B98FE0EF
:2004600087B980EC8BB986EA8AB985E08093C40080E48CBD1DBC0DB40EB408958DB780959E
:20048000E0E0F1E02FEF32E0281B3109E217F30710F41192FBCF109290011092A80110929A
:2004A000A60181E08093A7011092BE011092BD011092BF011092C1011092F1011092F501C6
:2004C0001092F6011092F7011092F8011092F9011092FA011092850108951F9395E5909301
:2004E000420180914201809341018091410180934001909345018091450180934401809140
:200500004401809343018FEF809347018091470180934601809187018093480116E3109322
:20052000490110934A0110934B0187E080934C0181E080934D0110924E018091FC018093F9
:200540004F0190935001909351013DD0109381018091FC0180938201109383011F91089518
:2005600020E0281750F49FE00000000000000000915097FFF9CF2F5FF4CF0895CF93D6D143
:200580005D9AC0E02C2F00002F5F2F3FE1F740E050E020E4CA0187709070892B19F4CC0FE3
:2005A0004899C16021504F5F5F4F27FFF3CF01D28C2F9927CF910895E1DF8F77803608F0C5
:2005C0008C5399270895ECE4F1E020E090914C01923020F0819128279150FACF20830895B3
:2005E000FF920F931F93CF93E7DF80939201C1E081E0F82E0C2F11270E561E4FDDDFF80127
:20060000808320E0D801E22FFF27EE56FE4F9C918081981721F02F5FC217A9F702C0FF2060
:2006200049F7CF5FC43120F3CF911F910F91FF90089580918601806480938601BAD188D36C
:200640001092C0001092C1001092C20080E290E09093890080938800809190018823E1F337
:20066000109290018091010181FFF6CF8091FC0180934A0180914D01846080934D01A3DF5D
:20068000809190018823E1F3109290018091010181FFF6CF8091010182FFF2CF84E38093DF
:2006A0004C019FEFE2E5F1E083E09193815087FFFCCF95E5E6E5F1E088E29193815087FF23
:2006C000FCCF81DF8091860180618093860108958091860185FFDCC08091A70184FF12C079
:2006E00080919001882371F08091010184FF0AC01092900180914D01877F80934D0180E291
:200700008093A70180914E0180FF31C080914E0182FF04C084E080934E0102C010924E0130
:200720008091F101882381F48091C30181FF50C0A4ECB1E0E1E4F1E090E18D91858B9150FA
:20074000319697FFFACF0FC08091DA0181FF40C0ABEDB1E0E1E4F1E090E18D91858B9150F9
:20076000319697FFFACF80914E0182602FC080914E0181FF02C083E001C081E080934E0199
:200780008091F101882381F48091C30181FF20C0A4ECB1E0E1E4F1E090E18D9184A79150AF
:2007A000319697FFFACF0FC08091DA0181FF10C0ABEDB1E0E1E4F1E090E18D9184A79150AE
:2007C000319697FFFACF80914E01846080934E018091F1018823B9F48091C30183FF37C0A4
:2007E0008091F801882399F58091D5018530B9F0A5EDB1E0E2E5F1E093E08D918193915030
:2008000097FFFBCF1AC08091DA0183FF20C08091F8018823E1F48091EC01853021F480E896
:200820008093850114C0ACEEB1E0E2E5F1E093E08D918193915097FFFBCF80914E0188605A
:2008400080934E011092F90181E08093F8018091F801813091F48091F901893121F483E0B0
:200860008093F8010AC080914E01886080934E018091F9018F5F8093F9018091FA0188233B
:2008800029F080914E01806880934E019CDE08958091A70181FF17C08091010184FF45C0D3
:2008A00080914D01877F80934D018091A801809351018091A8018F5F8093A80184DE84E029
:2008C0008093A70108958091A70182FF16C08091A801809351018091A8018F5F8093A8012D
:2008E00072DE8091A80184FF20C01092A7018091860180628093860108958091A70180FF58
:2009000014C0A2E9B1E0E0E4F1E093E18D91828B9150319697FFFACF80914D018860809352
:200920004D0151DE82E08093A7010895299A5A9A419A5D9828985C985998549A0895982F02
:20094000299A59985C98419834E360FF0BC080919101880F80939101309191013167892F53
:20096000855E0FC0892F845E20EA98E05C9827FF02C0599A01C05998220F5C9A915097FF8A
:20098000F5CF8068232F3327322F2227280F311D9FE05C9837FF02C0599A01C05998220F8F
:2009A000331F5C9A915097FFF4CF5C985998419A08955D98289829985A9841985C98599832
:2009C00008951F920F920FB60F9211242F933F934F935F936F937F938F939F93AF93BF9329
:2009E000CF93EF93FF93C0918801CF5F8C2F9927AA27BB27FC013197E830F10508F094C12B
:200A0000E65EFF4F09948091860185FF3FC08091A601E82FFF27EE56FE4F8081809387016A
:200A20008091A6018F5F8093A6018091A6018431C1F51092A6018091A70185FF12C08091CA
:200A4000BF01E82FFF27EE56FE4F8091C00180831092A7018091BF01E82FFF27E755FE4F52
:200A600010828091BD019091BE0101969093BE018093BD018091BD019091BE01885E934083
:200A800081F41092BE011092BD010BC080918701815E8093870180918701853610F010924C
:200AA000870161E0809187014ADF80E48093C00088E08093C1008091880090918900855917
:200AC0009E4F909389008093880080918701809348018091860184FDFBDD80914C01845FBB
:200AE0008093890121C18091880090918900805F9A4F909389008093880010928A0186E48E
:200B00008093C200289A88E28093C10085E58093C6008093C60008C109DF80918800909179
:200B200089008B5B9F4F49C08091860185FF0DC08091BD019091BE01892B39F48091A6011E
:200B4000E82FFF27E755FE4F108210928B0110928C011092900110928D0160E080918701A4
:200B6000EEDE80918800909189008C5E9E4F90938900809388005498D7C08091880090910B
:200B80008900895A9F4F90938900809388005D9A8091870180938001C7C010928D01109237
:200BA000C00080E98093C10086E48093C20080918800909189008C599B4F90938900809328
:200BC0008800B2C01092C0001092C1001092C200F0DEC0E0809188009091890084559F4F7A
:200BE000909389008093880080918C018F3FE1F580918D018823C1F521E02093900188B1EE
:200C000098E0892788B9C093FB018091020180FF05C08091020182FD09C004C08091020190
:200C200081FD04C08091F701882311F02093F5018091020183FF0AC08091FA01882361F4A8
:200C400081E08093F6018093FA0106C08091FA01882311F01092FA018091020187FF22C084
:200C600082E08093F8011EC081E08093F7018091860184FF0AC08091FB018F5F8093FB01CD
:200C80008091FB018F3F09F45F9A8091860185FF09C08091A601E82FFF27E755FE4F80811F
:200CA0008F5F80838091860185FF3EC08091A7018823B9F58091A601E82FFF27E755FE4F99
:200CC0008081833070F180914D01886080934D018091A6018093BF018091A60180934F01B1
:200CE0008091A601E82FFF27EE56FE4F8081835E8093C0018091C0018F3528F08091C00138
:200D00008F558093C0018091C001809350018091C0019091A601890F8093510180E18093DA
:200D2000A70181E08093C101C0938801FF91EF91CF91BF91AF919F918F917F916F915F91A9
:200D40004F913F912F910F900FBE0F901F90189510928500109284001092800082E08093D8
:200D6000810080936F0086BB08951092850010928400109280001092820082E086BB1092BA
:200D80006F0083E0809381000895DEBBDFB7DABDCBBDD1E0C0918A01C05CD881D093C600D7
:200DA000CF53C0938A01C83009F42998D0918901DC1731F4D0E4D093C000D8E4D093C100C3
:200DC000CBB5DAB5DFBFDEB31895DEBBDFB7DABDD0E0D093C000D093C100D093C2005A9854
:200DE00028984198DAB5DFBFDEB318959EBBEABDFBBDFFB7F8BD90918C019430B1F0E0E8F1
:200E0000F1E0E90FF081E091C600FE1771F5939590938C01943059F5E0918400E0938E0105
:200E2000E0918500E0938F0122C09091C600F1E0E0918B019083E395EF73E0938B01F091B5
:200E40008D01F927F0938D01909100019E1779F49FEF90938C0190E09093C1009093C20018
:200E60005A985D984198299802C010928C01F8B5FFBFFBB5EAB59EB31895F999FECFB2BD7A
:200E8000A1BDF89A119600B40895FFFFFFFFFFFFFFFFFFFFFFFFFFFFFFFFFFFFFFFFFFFF80
:200EA0000FEFFFFFFFFFFFFFFFFFFFFFFFFFFFFFFFFFFFFFFFFFFFFFFFFFFFFFFFFFFFFF52
:200EC0000FEFFFFFFFFFFFFFFFFFFFFFFFFFFFFFFFFFFFFFFFFFFFFFFFFFFFFFFFFFFFFF32
:200EE0000FEFFFFFFFFFFFFFFFFFFFFFFFFFFFFFC8030300C9EEFF00CA000000FFFFFFFFB8
:200F00008091BC008823E4F7089500E010E068018DE38093B80086E68093BA0084EC8093B1
:200F2000BC00EEDF8091B900887F803609F0FFCF84EC8093BC00E4DF8091B900887F80384F
:200F400009F0FFCF8091BB00182F84EC8093BC00D7DF8091B900887F803809F0FFCF809161
:200F6000BB00082FC8018F739070892B09F0FFCF8FE00030180708F0FFCFE80184EC809349
:200F8000BC00EE24FF248FE3B82EBADF8091B900887F803891F4E0FC04C08091BB00C82EFF
:200FA0000DC08091BB00D82E81E00601FE0180935700E8951124229601C0FFCF84EC809345
:200FC000BC00BA940894E11CF11CB7FEDECF98DF8091B900887F803A09F0FFCF84EC8093B3
:180FE000BC0083E0F80180935700E89585E0F80180935700E89595CF51
:00000001FF
